:100000000C9472000C949A000C949A000C949A0030
:100010000C949A000C949A000C949A000C949A00F8
:100020000C949A000C949A000C949A000C949A00E8
:100030000C949A000C949A000C949A000C949A00D8
:100040000C94A50B0C949A000C94150C0C94EF0BCB
:100050000C949A000C949A000C949A000C949A00B8
:100060000C94470C0C949A00005EBCE2613FDD8367
:10007000C29C7E20A3FD1F41009D23BE46DB65F888
:100080008C11AF32CA57E974000000002400270029
:100090002A0000000000250028002B0000000008B6
:1000A000000201000003040700000000000000003F
:1000B00000000000230026002900040404040404B6
:1000C0000404020202020202030303030303010207
:1000D00004081020408001020408102001020408D6
:1000E0001020660D11241FBECFEFD8E0DEBFCDBFBC
:1000F00024E0AAE9B2E001C01D92AC33B207E1F7F7
:1001000012E0A0E0B1E0ECE9FFE202C005900D9240
:10011000AA39B107D9F710E0C2E7D0E004C02197AF
:10012000FE010E94C617C137D107C9F70E94FB0D17
:100130000C94CC170C940000833081F028F48130AB
:1001400099F08230A9F008958730A9F08830C9F07D
:100150008430B1F4809180008F7D03C08091800055
:100160008F7780938000089584B58F7784BD08953C
:1001700084B58F7DFBCF8091B0008F778093B000E6
:1001800008958091B0008F7DF9CF1F93CF93DF93B7
:10019000282F30E0F901E456FF4F8491F901E25332
:1001A000FF4FD491F901E654FF4FC491CC23A9F03D
:1001B000162F81110E949C00EC2FF0E0EE0FFF1F24
:1001C000EE56FF4FA591B4918FB7F894EC911111B1
:1001D00008C0D095DE23DC938FBFDF91CF911F91B4
:1001E0000895DE2BF8CFCF93DF9390E0FC01E2532C
:1001F000FF4F249186549F4FFC0184918823C9F0BE
:1002000090E0880F991FFC01E857FF4FA591B4912A
:10021000FC01EE56FF4FC591D49161110DC09FB7FF
:10022000F8948C91209582238C93888128232883AD
:100230009FBFDF91CF910895623051F49FB7F8943A
:100240003C91822F809583238C93E8812E2BEFCFD6
:100250008FB7F894EC912E2B2C938FBFEACF1F937E
:10026000CF93DF93182FEB0161E00E94F3002097FA
:1002700039F460E0812FDF91CF911F910C94C5007C
:10028000CF3FD10511F461E0F5CFE12FF0E0E45666
:10029000FF4FE491E33031F140F4E130B1F0E2306E
:1002A000E1F0C038D1057CF7E4CFE73029F1E83040
:1002B00059F1E430B1F78091800080628093800032
:1002C000D0938B00C0938A0004C084B5806884BD3D
:1002D000C7BDDF91CF911F91089584B5806284BD21
:1002E000C8BDF7CF80918000806880938000D09354
:1002F0008900C0938800EDCF8091B0008068809322
:10030000B000C093B300E5CF8091B00080628093CD
:10031000B000C093B400DDCF3FB7F89480915D0387
:1003200090915E03A0915F03B091600326B5A89BF6
:1003300005C02F3F19F00196A11DB11D3FBFBA2F77
:10034000A92F982F8827BC01CD01620F711D811D37
:10035000911D42E0660F771F881F991F4A95D1F7BC
:1003600008958F929F92AF92BF92CF92DF92EF92B9
:10037000FF926B017C010E948C014B015C01C11456
:10038000D104E104F104B9F00E948C0168197909E3
:100390008A099B09683E73408105910580F321E03D
:1003A000C21AD108E108F10888EE880E83E0981E91
:1003B000A11CB11CE4CFFF90EF90DF90CF90BF90D5
:1003C000AF909F908F9008952FB7F8946091590344
:1003D00070915A0380915B0390915C032FBF089545
:1003E00008950895AF92BF92CF92DF92EF92FF925D
:1003F0000F931F93CF93DF936C017B018B01040F4D
:10040000151FEB015E01AE18BF08C017D10759F0E8
:100410006991D601ED91FC910190F081E02DC6012A
:100420000995892B79F7C501DF91CF911F910F9124
:10043000FF90EF90DF90CF90BF90AF900895FC01B8
:10044000538D448D252F30E0842F90E0821B930B39
:10045000541710F0CF96089501970895FC01918DDF
:10046000828D981761F0A28DAE0FBF2FB11D5D96E2
:100470008C91928D9F5F9F73928F90E008958FEF84
:100480009FEF0895FC01918D828D981731F0828D38
:10049000E80FF11D858D90E008958FEF9FEF08958F
:1004A0000F931F930E94E4016093690370936A03A2
:1004B00080936B0390936C0381E693E00E94420269
:1004C00097FF1DC00E94E4010091690310916A0327
:1004D00020916B0330916C03601B710B820B930BAB
:1004E00000916503109166032091670330916803C2
:1004F0006017710782079307F8F28FEF9FEF1F9144
:100500000F910895FC01918D228D892F90E0805CE0
:100510009F4F821B91098F739927089581E693E07D
:100520000E94820221E0892B09F420E0822F0895A5
:1005300080E090E0892B29F00E948E0281110C94BA
:1005400000000895FC01A48DA80FB92FB11DA35A76
:10055000BF4F2C91848D90E001968F739927848FE3
:10056000A689B7892C93A089B1898C918370806406
:100570008C93938D848D981306C00288F389E02DA7
:1005800080818F7D80830895EF92FF920F931F9358
:10059000CF93DF93EC0181E0888F9B8D8C8D981336
:1005A0001AC0E889F989808185FF15C09FB7F89442
:1005B000EE89FF896083E889F9898081837080648E
:1005C00080839FBF81E090E0DF91CF911F910F91D9
:1005D000FF90EF900895F62E0B8D10E00F5F1F4FE8
:1005E0000F731127E02E8C8D8E110CC00FB607FCF7
:1005F000FACFE889F989808185FFF5CFCE010E9485
:10060000A202F1CFEB8DEC0FFD2FF11DE35AFF4F4E
:10061000F0829FB7F8940B8FEA89FB898081806212
:10062000CFCFCF93DF93EC01888D8823B9F0AA89CF
:10063000BB89E889F9898C9185FD03C0808186FD9D
:100640000DC00FB607FCF7CF8C9185FFF2CF8081EC
:1006500085FFEDCFCE010E94A202E9CFDF91CF91BD
:100660000895DC0180E0615090F09D919827E92F7A
:10067000EF70F0E0E859FF4F2491E92FE295EF7019
:10068000F0E0E858FF4FE491822F8E27ECCF0895D9
:10069000DC012C911196ED91FC91F8948181822BD3
:1006A00081839281322F30959323928387E090E06B
:1006B0000197F1F781818323818383E290E00197A1
:1006C000F1F790817894EFECF0E03197F1F7922315
:1006D00081E009F480E00895FC0190810180F281BD
:1006E000E02D292F209560FF14C0F8948281822389
:1006F00082838181892B8183A3E2B0E01197F1F796
:100700008281982B9283789487ED90E00197F1F79E
:100710000895F8948281822382838181892B818349
:10072000AFEFB0E01197F1F78281982B9283789424
:100730008FE090E0EBCFDF92EF92FF920F931F9349
:10074000CF93DF93EC01D62EE42E08E010E0FF24D7
:10075000F39461E08D2D8F2109F460E0CE010E94B9
:100760006C03FF0C01501109A1F7E11010C0F894BF
:10077000E981FA8191818881809589238183E9814A
:10078000FA81928188818095892382837894DF9190
:10079000CF911F910F91FF90EF90DF900895EF920E
:1007A000FF920F931F93CF93DF938C017B0140E067
:1007B00065E50E949B03E70188E0E80EF11C699162
:1007C00040E0C8010E949B03CE15DF05C1F7DF9111
:1007D000CF911F910F91FF90EF900895FC019081B0
:1007E0000180F281E02DF8948181292F20958223C8
:1007F000818378943DE743E050E0315029F1DA01FC
:100800001197F1F780818923C1F3F89482818223C3
:1008100082838181892B81837894ABE7B7E011973C
:10082000F1F7F894818182238183A3E1B1E01197EC
:10083000F1F78081982381E009F080E07894E3E685
:10084000F6E03197F1F7089580E008956F927F9276
:100850008F929F92AF92BF92CF92DF92EF92FF92D0
:100860000F931F93CF93DF938C01EB0180911304BF
:10087000909114040E94EE03882309F43FC0B8014C
:1008800080911304909114040E94CF0340E06EEB1A
:1008900080911304909114040E949B037E016E01C9
:1008A00089E0C80ED11C8E01A0901304B0901404EE
:1008B00088E0882E912C712C66246394C5010E94D7
:1008C000480381117628660CE1E08E1A9108B1F791
:1008D000F80171928F01CE16DF0631F78091130473
:1008E000909114040E94EE03813041F4F70181914C
:1008F0007F01811105C0E017F107C1F790E008C042
:1009000068E0CE010E94310391E028852813F6CFDC
:10091000892FDF91CF911F910F91FF90EF90DF9082
:10092000CF90BF90AF909F908F907F906F900895E1
:100930008F929F92AF92BF92CF92DF92EF92FF92EF
:10094000CF93DF9300D000D01F92CDB7DEB7809158
:100950001304909114040E94EE0340E06CEC80912B
:100960001304909114040E949B0340910A0464E4D0
:1009700080911304909114040E949B030E94E4014F
:100980006B017C0180910E0481111EC081E089837E
:10099000CA82DB82EC82FD8229813A814B815C81B3
:1009A0006D8170E080E090E00F900F900F900F90BD
:1009B0000F90DF91CF91FF90EF90DF90CF90BF909D
:1009C000AF909F908F90089580910F048823C1F07D
:1009D00080910A04811114C0809113049091140431
:1009E0000E944803813091F20E94E4016C197D0954
:1009F0008E099F096E3E72408105910568F3C6CF4E
:100A0000E0910D04E9508EEE92E0E33038F4F0E02E
:100A1000EE0FFF1FE254FE4F808191814C01B12CFB
:100A2000A12C80910B04882329F060E080910C04B4
:100A30000E94C500C501B4010E94B10180910B0460
:100A4000882309F4A3CF61E080910C040E94C500C3
:100A50009DCF08952091DB02260F3327331F2132CB
:100A60003105ECF420912403FC0190E080E0243077
:100A700069F082E00895A091DB022191AC01455418
:100A80005D4FA40FB52FB11D2C930196861798F3D7
:100A90008091DB02680F6093DB0280E0089581E0C3
:100AA00008951092240381E0809323031092FE02A4
:100AB00061E082E10E94C50061E083E10E94C5001F
:100AC000E9EBF0E080818E7F808380818D7F808361
:100AD00088E48093B80085E48093BC000895CF93A8
:100AE000DF9391E09093BA028823B9F0C091B800E7
:100AF000D091BA008091BC008A7B8093BC0060E0FA
:100B000082E10E94C50060E083E10E94C5000E946E
:100B10005105D093BA00C093B800DF91CF910895EA
:100B20000895E091530380915203E81730F4F0E008
:100B3000E656FD4F808190E008958FEF9FEF089576
:100B400090915303809152032FEF3FEF981748F491
:100B5000E92FF0E0E656FD4F208130E09F5F909353
:100B60005303C90108958091520390915303891B47
:100B7000990B0895CF92DF92EF92FF920F931F93FC
:100B8000CF93DF937C01CB018A0120912A0322239A
:100B900089F0EB016B01C40ED51ECC15DD0569F0A3
:100BA0006991D701ED91FC910190F081E02DC70191
:100BB0000995F3CF642F0E942A05C801DF91CF91D8
:100BC0001F910F91FF90EF90DF90CF900895CF93FA
:100BD000DF931F92CDB7DEB7698320912A032223CA
:100BE000F9F020915003203258F021E030E0FC0170
:100BF0003383228390E080E00F90DF91CF910895BE
:100C000080915103E82FF0E0E55DFC4F99819083DE
:100C10008F5F809351038093500381E090E0ECCF8D
:100C200061E0CE0101960E942A05F7CFCF92DF92B4
:100C3000EF92FF920F931F93CF93DF93FC01C48138
:100C400021E020932A03C0934B031092510310928A
:100C500050038485682B8EEF93E00E94E705D091C6
:100C60005003D13208F092C00E948C016B017C01CC
:100C700080912403811165C082E08093240381E088
:100C8000809323038FEF8093220310922103D0934C
:100C90002003ABE2B3E0E0E0F3E080E0D81385C0EE
:100CA0001092FF028091FF02CC0FC82BC093FF026D
:100CB0008091FE02813009F07CC01092FE020E94F9
:100CC0008C016B017C018091FF028093BB008091BD
:100CD000260390912703A0912803B0912903892B23
:100CE0008A2B8B2B99F00E948C0100912603109186
:100CF000270320912803309129036C197D098E095F
:100D00009F090617170728073907E0F18091BC00F3
:100D100083FDD9CF85EC8093BC000E948C016B01D0
:100D20007C0180912403823009F445C08091220324
:100D30008F3F61F180912203803241F18091220343
:100D400025C08091260390912703A0912803B0919C
:100D50002903892B8A2B8B2B09F48ACF0E948C01C3
:100D60000091260310912703209128033091290335
:100D70006C197D098E099F0906171707280739077F
:100D800008F076CF809125030E946F0510925103E1
:100D90001092500310922A03DF91CF911F910F916F
:100DA000FF90EF90DF90CF9008959D9191938F5F8A
:100DB00075CF85EEB0CF8091260390912703A09147
:100DC0002803B0912903892B8A2B8B2B09F4A9CFF7
:100DD0000E948C0100912603109127032091280383
:100DE000309129036C197D098E099F090617170791
:100DF0002807390708F095CFC5CF90E080E0089527
:100E00002F923F924F925F926F927F928F929F921A
:100E1000AF92BF92CF92DF92EF92FF920F931F9308
:100E2000CF93DF9300D000D000D0CDB7DEB76B01F9
:100E30007C015A8349838901FA0160817181072EFF
:100E4000000C880B990B0E941F15A70196010E94A8
:100E50006B1787FD0AC0F80160817181072E000CB5
:100E6000880B990B0E941F158EC0E981FA81648955
:100E70007589072E000C880B990B0E941F15A7017E
:100E800096010E94181518160CF0A2C029803A800D
:100E90001E821D82F101619171911F01072E000CCC
:100EA000880B990B0E941F154B015C01AC019B0143
:100EB000C701B6010E946B172D813E812E5F3F4F07
:100EC0003A83298387FD78C0F10160817181072E03
:100ED000000C880B990B0E941F152B013C01AC01E3
:100EE0009B01C701B6010E94181518160CF464C0C6
:100EF0002D813E81200F311FF9010190F081E02DFD
:100F0000FE83ED8329813A81020F131FF80160816E
:100F100071812D813E81621B730B072E000C880BA3
:100F2000990B0E941F1569837A838B839C83A5018B
:100F30009401C701B6010E9456166B017C01A50100
:100F40009401C301B2010E9456169B01AC01C70176
:100F5000B6010E94C3169B01AC0169817A818B8125
:100F60009C810E947E156B017C01ED81FE81BF0199
:100F7000FF0F880B990B0E941F159B01AC01C70145
:100F8000B6010E94571626960FB6F894DEBF0FBE24
:100F9000CDBFDF91CF911F910F91FF90EF90DF9028
:100FA000CF90BF90AF909F908F907F906F905F9009
:100FB0004F903F902F90089529813A813E832D8351
:100FC0002431310509F066CF60E070E0CB01DBCF62
:100FD000F8016489758942CFBF92CF92DF92EF9278
:100FE000FF920F931F93CF93DF93EC01B62EC72E82
:100FF0008D85811105C0CE010E94EE0381110EC0C6
:101000001B861D861C8680E0DF91CF911F910F917A
:10101000FF90EF90DF90CF90BF90089540E060EF99
:10102000CE010E949B0301E0E12CD12C11E0CE0106
:101030000E944803F82ECE010E94480391E0F91265
:1010400018C0813099F51134D8F2DB86D11002C076
:1010500081E08D878B81882399F22396EB2DFC2DDF
:10106000CF01089629912193E817F907D9F781E074
:10107000CBCFEE2DF0E0F8120FC08B851817A0F43F
:10108000DE01AE0FBF1F13968C91802379F4F12CF3
:10109000193008F41C87D12EEC0FFD1F8381902F8F
:1010A0009095892383830AC08113F1CFFE01EE0D51
:1010B000F11D8381802B8383FF24F3946F2DCE0158
:1010C0000E946C031F5F000F11F4E39401E087E0BE
:1010D0008E1508F0ACCFB7CFCF92DF92EF92FF9290
:1010E0000F931F93CF93DF93CDB7DEB761970FB602
:1010F000F894DEBF0FBECDBF80911104811113C0E3
:1011000060E070E08EEF92EC61960FB6F894DEBF6F
:101110000FBECDBFDF91CF911F910F91FF90EF9048
:10112000DF90CF900895E0911304F091140413869A
:1011300015861486128611861086178216821582ED
:1011400014821382BE01665F7F4F809113049091D9
:1011500014040E94EC07882399F267E0CE010A96F6
:101160000E94310399898913CBCFBE016F5F7F4FF6
:10117000CE010A960E942604882311F29A81C12C7E
:10118000D12C760197FF06C0C12CD12CF8EFEF2EA1
:10119000FF24FA944A8589814B33E1F52D8127FF9D
:1011A00039C080FDADCF082F10E030E020E073E0C3
:1011B000000F111F221F331F7A95D1F7007E177081
:1011C00022273327892F90E0B0E0A0E0EBE0880FE2
:1011D000991FAA1FBB1FEA95D1F7802B912BA22B39
:1011E000B32B8C019D010C291D292E293F29013883
:1011F00054EE15075FEF250735070CF481CFC901C1
:10120000B8010E941F1520E030E040E05CE30E943E
:101210007E157ACF092F10E0102F0027110F110F24
:10122000110F28E0829FB0011124062B172B012EED
:10123000000C220B330B0C291D292E293F29483283
:1012400069F4803531F4953091F68F818C3079F6E0
:1012500057CF8F3F61F6973051F652CF403139F674
:101260006885662321F270E08F81AB01481B51092C
:10127000CA019695982F8827979587950E9475178C
:10128000CB01770FAA0BBB0B53E0000F111F221FDE
:10129000331F5A95D1F70078277033270052110970
:1012A00021093109800F911FA21FB31F97018601E9
:1012B000082B192B2A2B3B2B9ACF0F931F93CF93DD
:1012C0008C01C62F0E9416066C2F6460C8010E9414
:1012D00016066C2F6B7FC8010E94160683EC90E007
:1012E0000197F1F7CF911F910F9108950F931F93DD
:1012F000CF93DF938C01D62FC42F607F642B0E9485
:101300005D0980E1D89FB00111246C2BC801DF91E9
:10131000CF911F910F910C945D0941E00E947609D5
:1013200081E090E00895CF93DF93CDB7DEB72897A3
:101330000FB6F894DEBF0FBECDBF98E0E8E4F1E051
:10134000DE01119601900D929A95E1F79091370484
:10135000981708F48FEF90E0880F991F21E030E094
:101360002C0F3D1F820F931FFC016081606840E0DD
:101370008FE294E028960FB6F894DEBF0FBECDBF83
:10138000DF91CF910C9476090F931F93CF93DF9346
:101390008B0198E0899FB0011124606440E08FE2E6
:1013A00094E00E947609E801085F1F4F69918FE27F
:1013B00094E00E948D09C017D107C1F7DF91CF914A
:1013C0001F910F91089540E061E08FE294E00E9448
:1013D00076098BE39FE10197F1F780913804882328
:1013E00019F080E00C9493090895FB01019000200E
:1013F000E9F73197AF01461B570BDC01ED91FC91EA
:101400000280F381E02D09948F929F92AF92BF9258
:10141000EF92FF920F931F93CF93DF93CDB7DEB779
:10142000A1970FB6F894DEBF0FBECDBF7C01FA01C5
:10143000CB0119A2223008F42AE08E010F5D1F4F64
:10144000822E912CB12CA12CBF01A50194010E94E8
:101450008917F901CA016A300CF5605DD8016E93F5
:101460008D01232B242B252B79F790E080E010971A
:1014700021F0BD01C7010E94F509A1960FB6F894AD
:10148000DEBF0FBECDBFDF91CF911F910F91FF90B7
:10149000EF90BF90AF909F908F900895695CDECFE2
:1014A000CF92DF92EF92FF926C01990FEE08FF0846
:1014B000F7FE18C041E06DE28FE294E00E947609E9
:1014C00044275527BA014C195D096E097F092AE0A6
:1014D0008FE294E00E94040A0196FF90EF90DF9063
:1014E000CF9008952AE0B701A6018FE294E0FF9023
:1014F000EF90DF90CF900C94040A2F923F924F927E
:101500005F926F927F928F929F92AF92BF92CF9293
:10151000DF92EF92FF921F93CF93DF93EC016A016A
:101520007B01722EAB019601CB01B6010E947017B0
:1015300064EF71E0811126C046015701E894B7F8C5
:101540002FEF3FEF4FE75FE7C501B4010E9470172F
:1015500081110CC02FEF3FEF4FE75FE7C501B401EA
:101560000E94181568EF71E0181664F02FEF3FEF36
:101570004FE75FE4C701B6010E946B171816B4F479
:101580006CEF71E0CE01DF91CF911F91FF90EF9052
:10159000DF90CF90BF90AF909F908F907F906F9093
:1015A0005F904F903F902F900C94F5092FEF3FEFF5
:1015B0004FE75FECC701B6010E94181587FDE0CF29
:1015C00020E030E0A901C701B6010E941815312CB6
:1015D000212C87FF0DC0E881F9810190F081E02D79
:1015E0006DE2CE0109951C01F7FAF094F7F8F0943A
:1015F00010E060E070E080E09FE3711641F020E0D1
:1016000030E040E251E40E94C3161F5FF6CFA7010D
:1016100096010E9457162B013C010E943C174B017A
:101620005C012AE0BC01A401CE010E94040A7C01F5
:10163000E20CF31C1123E1F1C501B4010E941D1558
:101640009B01AC01C301B2010E9456164B015C0123
:10165000E881F9810190F081E02D6EE2CE010995DB
:10166000E80EF91E115020F120E030E040E251E494
:10167000C501B4010E947E152B013C010E943C175C
:101680004B01B12CA12C2AE0B501A401CE010E948E
:10169000040AE80EF91EC501B4010E941D159B0144
:1016A000AC01C301B2010E9456164B015C01DACFB6
:1016B000C701DF91CF911F91FF90EF90DF90CF9006
:1016C000BF90AF909F908F907F906F905F904F9062
:1016D0003F902F9008950C94F50985ED8093BC0000
:1016E0008091260390912703A0912803B0912903AC
:1016F0000796A11DB11D23E0B695A79597958795EF
:101700002A95D1F72091BC0024FD03C01092240338
:10171000089540912603509127036091280370910A
:101720002903452B462B472B69F30097A105B105EB
:1017300041F02AE22A95F1F700C00197A109B10909
:10174000E1CF809125030C946F051F920F920FB685
:101750000F9211242F933F938F939F93AF93BF9337
:101760008091590390915A03A0915B03B0915C035F
:101770003091580323E0230F2D3758F50196A11D12
:10178000B11D209358038093590390935A03A0935B
:101790005B03B0935C0380915D0390915E03A09125
:1017A0005F03B09160030196A11DB11D80935D039D
:1017B00090935E03A0935F03B0936003BF91AF91DA
:1017C0009F918F913F912F910F900FBE0F901F907F
:1017D000189526E8230F0296A11DB11DD2CF1F92A6
:1017E0000F920FB60F9211242F933F934F935F9355
:1017F0006F937F938F939F93AF93BF93EF93FF93D9
:1018000081E693E00E94A202FF91EF91BF91AF9118
:101810009F918F917F916F915F914F913F912F9108
:101820000F900FBE0F901F9018951F920F920FB63A
:101830000F9211242F938F939F93EF93FF93E09137
:101840007103F09172038081E0917703F091780346
:1018500082FD1BC0908180917A038F5F8F732091EE
:101860007B03821741F0E0917A03F0E0EF59FC4FDF
:10187000958F80937A03FF91EF919F918F912F9194
:101880000F900FBE0F901F9018958081F4CF1F927C
:101890000F920FB60F9211242F933F934F935F93A4
:1018A0006F937F938F939F93AF93BF93EF93FF9328
:1018B0008091B900887F803609F44AC0F0F58832FB
:1018C00009F4A7C018F5803109F49BC0B8F4882347
:1018D00009F4F9C0883009F494C0FF91EF91BF91E9
:1018E000AF919F918F917F916F915F914F913F91B8
:1018F0002F910F900FBE0F901F901895883109F40B
:1019000088C0803251F78093220314C0803409F4D8
:101910009DC040F48033B9F38833F9F680932203F5
:1019200085ECB0C0803509F485C0883509F496C0CF
:10193000883499F60E946D0BD0CF883909F48CC099
:1019400038F5883729F050F4883611F0803729F6B9
:1019500083E0809324031092FD0257C0883809F475
:101960007BC0803919F0803809F0B7CF8091FD0233
:10197000803208F071C0E091FD0281E08E0F80930B
:10198000FD028091BB00F0E0E352FD4F80833DC03B
:10199000803B39F0E0F4803A09F479C0883A09F0E4
:1019A0009CCF84E0809324031092DC021092DB022F
:1019B000E0914E03F0914F0309958091DB02811174
:1019C0000FC081E08093DB021092BB0209C0803C13
:1019D00009F4A6CF883C09F4A3CF883B09F07DCF5A
:1019E000E091DC0281E08E0F8093DC02F0E0E554B0
:1019F000FD4F80818093BB009091DC028091DB02DF
:101A000029C08091FF028093BB0085EC8093BC00CD
:101A100064CF9091210380912003981758F5E091AD
:101A2000210381E08E0F80932103F0E0E050FD4F11
:101A30008081E9CFE091210381E08E0F8093210323
:101A40008091BB00F0E0E050FD4F80839091210336
:101A5000809120039817C8F285E8D8CFE091210340
:101A600081E08E0F809321038091BB00F0E0E05075
:101A7000FD4F80838091230381115CCF81E08093AF
:101A8000FE0284EA8093BC001092240326CF85ECEA
:101A90008093BC00109224038091FD02803230F4C8
:101AA000E091FD02F0E0E352FD4F10826091FD02F3
:101AB00070E0E0914C03F0914D038DED92E00995BB
:101AC0001092FD020ACF1092220334CFE1E6F3E038
:101AD0001382128288EE93E0A0E0B0E084839583C5
:101AE000A683B78328EC31E03183208325EC30E0F6
:101AF0003587248724EC30E03787268720EC30E0D8
:101B0000318B208B21EC30E0338B228B22EC30E0C8
:101B1000358B248B26EC30E0378B268B118E128E82
:101B2000138E148EEEEFF3E013821282848395837A
:101B3000A683B7838AED91E091838083EFE2F4E09E
:101B4000138212828CEE91E091838083118687E26A
:101B5000848380E1828782E08387148660E087E067
:101B60000E94F300E5EDF0E0E491A1E2B4E0EC9333
:101B7000E1ECF0E0E491F0E0EE0FFF1FE055FF4FE5
:101B80008591949112969C938E9311971B961C921B
:101B90001B971D961C921D971C961C921C971A96BB
:101BA0001C921A9719961C92199718961C921897BE
:101BB00017961C92179716961C92169715961C92BC
:101BC000159714961C92149713961C921397EAE09B
:101BD000F4E017821086108289E0838381E0848399
:101BE000858386831182168A158A8FEF838B148AE8
:101BF000B287A1870895CF93DF93CDB7DEB76F97F4
:101C00000FB6F894DEBF0FBECDBF789484B5826066
:101C100084BD84B5816084BD85B5826085BD85B590
:101C2000816085BD80916E00816080936E0010920E
:101C30008100809181008260809381008091810089
:101C4000816080938100809180008160809380001A
:101C50008091B10084608093B1008091B000816078
:101C60008093B00080917A00846080937A008091A4
:101C70007A00826080937A0080917A0081608093FC
:101C80007A0080917A00806880937A001092C10077
:101C9000E0917103F091720382E08083E0916D0323
:101CA000F0916E031082E0916F03F09170038FEC5E
:101CB000808310927903E0917503F091760386E0BA
:101CC0008083E0917303F09174038081806180834D
:101CD000E0917303F0917403808188608083E091C8
:101CE0007303F0917403808180688083E0917303B3
:101CF000F091740380818F7D808361E08BE00E948E
:101D0000F30061E08AE00E94F30061E089E00E9454
:101D1000F30061E083E00E94F30061E086E00E944E
:101D2000F30062E08CE00E94F30060E08BE00E9430
:101D3000C50060E08AE00E94C50060E089E00E9482
:101D4000C50060E083E00E94C50060E086E00E947C
:101D5000C500109253031092520310925103109237
:101D600050030E94510580EF91E090934F038093C0
:101D70004E0381EF91E090934D0380934C031092BA
:101D8000340480913A04823018F098E0909334043F
:101D90008093370462E370E080E090E00E94B1013C
:101DA00060913B048FE294E00E94160668EE73E0B7
:101DB00080E090E00E94B10160E38FE294E00E9435
:101DC0005D090BE416E4C8010197F1F760E38FE2C7
:101DD00094E00E945D09C8010197F1F760E38FE28A
:101DE00094E00E945D0983E592E00197F1F760E2DB
:101DF0008FE294E00E945D0960913404606240E0EB
:101E00008FE294E00E94760984E08093350440E0FC
:101E10006CE08FE294E00E9476090E94E30982E080
:101E20008093360440E066E08FE294E00E947609F9
:101E300040E062E08FE294E00E9476098BE39FE14C
:101E40000197F1F788E080933B0460E08FE294E033
:101E50000E9416060E94E30968E371E080E00E9498
:101E6000C40960E371E081E00E94C40968E271E0A6
:101E700082E00E94C40960E271E083E00E94C4092C
:101E800068E171E084E00E94C40960E171E085E0EE
:101E90000E94C40968E071E086E00E94C40960E025
:101EA00071E087E00E94C40980E00E94930967E620
:101EB00072E08FE294E00E946B0B60E08FE294E0AE
:101EC0000E948D0960E072E08FE294E00E946B0B4B
:101ED00081E00E9493096CE372E08FE294E00E943B
:101EE0006B0B61E08FE294E00E948D096FE772E076
:101EF0008FE294E00E946B0B60E08FE294E00E941E
:101F00008D096EE072E08FE294E00E946B0B66E058
:101F10008FE294E00E948D0964E172E08FE294E028
:101F20000E946B0B64E08FE294E00E948D0913E045
:101F300001E0E0911304F0911404138615861486D1
:101F400012861186108617821682158214821382D9
:101F5000109211041092120462E370E080E090E0AD
:101F60000E94B101BE01665F7F4F80911304909182
:101F700014040E94EC07882309F47AC067E0CE01BC
:101F80000A960E94310399898913ECCF809111043C
:101F90008F5F809311048A85883231F008F04EC03B
:101FA000803111F08232F1F6809112048F5F8093BC
:101FB000120480910A04811128C080911304909129
:101FC00014040E94EE03BE01665F7F4F80911304EC
:101FD000909114040E94CF0340E064EB80911304BD
:101FE000909114040E949B03809113049091140417
:101FF0000E944803F82E80911304909114040E94CB
:10200000EE03F11002C000930A048A85803109F1C1
:10201000BE016F5F7F4FCE010A960E94260488237F
:1020200059F08D819A859B3311F487FD12C08F334F
:1020300091F058F48F31C1F080E00EC08B3309F479
:10204000B3CF823409F08ECFAFCF8F3579F08F3791
:1020500099F78CE001C08AE090910D04981708F080
:1020600081CF80930D047ECF89E0F6CF8BE0F4CF53
:1020700080911104811103C0115009F05ACF0E94C0
:1020800098042F8B388F498F5A8F6B8F0E946C0862
:102090006B017C0120E030E04EEF52EC0E941815FD
:1020A000882341F0C0924001D0924101E092420168
:1020B000F09243016CED75E080E090E00E94B10188
:1020C00081E693E00E948202181619060CF0CFC038
:1020D0000E945002FC0197FDC6C08D32910559F057
:1020E000C0970A9740F0EE32F10529F081E693E0BF
:1020F0000E942E02EDCF10E000E0412C512C20E890
:10210000622E2FE3722EC12CD12C7601E130F10525
:1021100049F1ED32F105C9F1EE32F105C1F1CF011E
:10212000C0970A97F8F4AAE0B0E0A70196010E94D0
:102130003C166F01FF0FEE08FF08C60ED71EE81E03
:10214000F91E20E3C21AD108E108F108112351F069
:102150002DEC3CEC4CEC5DE3C301B2010E947E151A
:102160002B013C0181E693E00E942E020E94500266
:10217000FC01C0970A9750F2EE32F10551F4112399
:1021800029F2102F01110BC01AC001E0EBCF11E0B2
:10219000E9CFE130F10509F4B9CF002341F0F09423
:1021A000E094D094C094C11CD11CE11CF11CC70167
:1021B000B6010E941F154B015C01112351F0C701AC
:1021C000B6010E941F15A30192010E947E154B01CA
:1021D0005C0120E030E040E252ECC501B4010E9415
:1021E0006B1787FD34C020E030E048EC52E4C501B5
:1021F000B4010E941815181654F18092440190926F
:102200004501A0924601B092470131E03093570357
:1022100067E172E081E693E00E946B0B409144011C
:1022200050914501609146017091470121E081E69E
:1022300093E00E947D0A6FE272E081E693E00E94E3
:10224000F50962E372E081E693E00E94F50981E618
:1022500093E00E948202181619064CF481E693E07E
:102260000E942E02F4CF812C912C5401C6CFE09015
:102270004401F0904501009146011091470120E092
:1022800030EC49E754E4B701C8010E9418158111E8
:1022900027C00E9498042A873B874C875D876E87FA
:1022A0000E946C087B018C0120E030E04EEF52EC84
:1022B0000E9418158111C6C2809155039091560352
:1022C0008A3091052CF40196909356038093550320
:1022D000E0904001F09041010091420110914301D2
:1022E0001092540320E030E048EA51E4B701C801FD
:1022F0000E94181587FFC4C220E030E048E452EC89
:10230000B701C8010E946B1718160CF0B9C222E978
:1023100031E048EA51E0B701C8010E9400074B01D3
:102320005C0120E030E0A9010E946B1720E030E062
:1023300040E05FE387FD95C2C501B4010E945716D6
:102340000E9435175B0126E631E04CE751E0B7010A
:10235000C8010E9400072B013C0120E030E0A901E8
:102360000E946B1720E030E040E05FE387FD7EC213
:10237000C301B2010E9457160E9435171B0120E5C8
:1023800031E04CE751E0B701C8010E9400072B0182
:102390003C0120E030E0A9010E946B1720E030E012
:1023A00040E05FE387FD67C2C301B2010E94571698
:1023B0000E9435176B0180915703882381F020E03C
:1023C00030E040E751E4B701C8010E946B1710925A
:1023D000570387FD04C0312C212CB12CA12CE8EA35
:1023E000F0E08491EAEDF0E08490E6ECF0E0949087
:1023F00091104DC20E94E30980E00E94930967E6B4
:1024000072E08FE294E00E946B0B66E08FE294E052
:102410000E948D0965E372E08FE294E00E946B0BED
:1024200061E08FE294E00E948D096FE772E08FE235
:1024300094E00E946B0B60E08FE294E00E948D09B3
:1024400060E472E08FE294E00E946B0B68EE73E050
:1024500080E090E00E94B101F1E0F0935403D12CB0
:10246000C12C312C212C96E0A92EB12C61E08BE0FF
:102470000E94C50061E08AE00E94C50061E089E039
:102480000E94C50061E083E00E94C50061E086E033
:102490000E94C5003701480181E693E00E94820254
:1024A00020915403181619060CF4A7C0E0904401BB
:1024B000F09045010091460110914701211142C25F
:1024C00020E030EC49E754E4B701C8010E94181538
:1024D000811127C00E9498042A8B3B8B4C8B5D8B0B
:1024E0006E8B0E946C087B018C0120E030E04EEF87
:1024F00052EC0E941815811116C2809155039091DB
:1025000056038A3091052CF40196909356038093DC
:102510005503E0904001F09041010091420110917B
:1025200043010E94E30980E00E94930963E472E0A2
:102530008FE294E00E946B0B64E08FE294E00E94D3
:102540008D0967E472E08FE294E00E946B0B61E01A
:102550008FE294E00E948D096FE772E08FE294E0D1
:102560000E946B0B60E08FE294E00E948D096BE4A7
:1025700072E08FE294E00E946B0BC5010E94500A4A
:102580006FE472E08FE294E00E946B0B81E00E94A6
:102590009309809155039091560361E572E00A9783
:1025A000ECF480915403882309F4D9C162E672E007
:1025B0008FE294E00E946B0B62E08FE294E00E9455
:1025C0008D0965E672E08FE294E00E946B0B66E095
:1025D0008FE294E00E948D096AE672E08FE294E057
:1025E0000E946B0B68EE73E080E090E00E94B10106
:1025F00021E0A21AB10809F04DCF60E08BE00E9403
:10260000C50060E08AE00E94C50060E089E00E94A9
:10261000C50060E083E00E94C50060E086E00E94A3
:10262000C50080915403811145C1121413040CF0AC
:1026300041C11C141D040CF03DC10E94E4012B019A
:102640003C0128EE33E0D1010E94AB176C8F7D8FE7
:102650008E8F9F8FB6018BE00E942F01B6018AE01A
:102660000E942F01B60189E00E942F01B60183E08C
:102670000E942F0161E086E00E94C5000E94E401F3
:1026800064197509860997092C8D3D8D4E8D5F8DD6
:10269000621773078407950708F08EC181E693E0FF
:1026A0000E948202181619060CF486C1809044011B
:1026B00090904501A0904601B090470120E030EC99
:1026C00049E754E4C501B4010E941815811127C0DF
:1026D0000E94980429833A834B835C836D830E9414
:1026E0006C084B015C0120E030E04EEF52EC0E94A0
:1026F0001815811154C180915503909156038A3069
:1027000091052CF401969093560380935503809085
:10271000400190904101A0904201B090430120E01F
:1027200030E040E751E4C501B4010E946B1787FF18
:1027300043C10E94E4014B015C0180E00E949309C7
:102740006EE672E08FE294E00E946B0B62E08FE233
:1027500094E00E948D0963E772E08FE294E00E94AA
:102760006B0B61E08FE294E00E948D0968E772E0F4
:102770008FE294E00E946B0B62E08FE294E00E9493
:102780008D0960E672E08FE294E00E946B0B81E0BD
:102790000E949309809155039091560361E572E080
:1027A0000A970CF044C06DE772E08FE294E00E945B
:1027B0006B0B62E08FE294E00E948D0967E472E0A7
:1027C0008FE294E00E946B0B61E08FE294E00E9444
:1027D0008D096FE772E08FE294E00E946B0B60E07E
:1027E0008FE294E00E948D096FE472E08FE294E042
:1027F0000E946B0B6CE272E08FE294E00E946B0B24
:10280000C501B401641975098609970928EE33E0FA
:1028100040E050E00E948917C101821B930B97FF93
:1028200002C090E080E00E94500A60E472E08FE213
:1028300094E00E946B0B68EC70E080E090E00E94F6
:10284000B1011CCF1092560310925503C701D80155
:102850008093400190934101A0934201B0934301C2
:102860003FCDC501B4010E9456166ACDC301B20125
:102870000E94561681CDC301B2010E94561698CD12
:10288000D12CC12C312C212CB12CA12C94CD811117
:102890000E949C00E92DF0E0EE0FFF1FE055FF4F76
:1028A000A591B4918C91882209F4A4CD1A141B042B
:1028B0000CF4DCCD0E94E30980E00E94930961E8FA
:1028C00072E08FE294E00E946B0B64E08FE294E090
:1028D0000E948D0969E272E08FE294E00E946B0B26
:1028E00080915503909156030A970CF47EC081E0C5
:1028F0000E94930961E572E08FE294E00E946B0B05
:1029000068EE73E080E090E00E94B10140E050E0AA
:10291000452B09F4D5CB0E948E02882309F4D0CB35
:102920000E940000CDCB1092560310925503C701B0
:10293000D8018093400190934101A0934201B0934C
:102940004301EFCD20E030EC49E754E4B701C80182
:102950000E9418158111E5CD73018401E2CD67E86D
:1029600072E08FE294E00E946B0B64E08FE294E0EF
:102970000E948D0969E272E08FE294E00E946B0B85
:1029800021E0A701B8018FE294E00E947D0A67E090
:102990008FE294E00E948D0960E372E01FCE1092F6
:1029A0005603109255038092400190924101A092EB
:1029B0004201B0924301B3CE70E060E08BE00E9430
:1029C0002F0170E060E08AE00E942F0170E060E07B
:1029D00089E00E942F0170E060E083E00E942F01F7
:1029E00060E086E00E94C50065CF21E0A701B80144
:1029F0008FE294E00E947D0A67E08FE294E00E94FB
:102A00008D0960E372E08FE294E00E946B0B81E03D
:102A10000E9493096AE872E08FE294E00E946B0BD7
:102A200066E08FE294E00E948D0966E972E064CF6F
:102A30000E945A1508F481E00895E89409C097FBB4
:102A40003EF490958095709561957F4F8F4F9F4F85
:102A50009923A9F0F92F96E9BB279395F6958795C9
:102A600077956795B795F111F8CFFAF4BB0F11F48C
:102A700060FF1BC06F5F7F4F8F4F9F4F16C0882333
:102A800011F096E911C0772321F09EE8872F762F69
:102A900005C0662371F096E8862F70E060E02AF0AA
:102AA0009A95660F771F881FDAF7880F9695879596
:102AB00097F90895990F0008550FAA0BE0E8FEEF6B
:102AC00016161706E807F907C0F012161306E407F2
:102AD000F50798F0621B730B840B950B39F40A26EB
:102AE00061F0232B242B252B21F408950A2609F4C9
:102AF000A140A6958FEF811D811D08950E9491151B
:102B00000C9402160E94F41538F00E94FB1520F078
:102B1000952311F00C94EB150C94F11511240C94E1
:102B200036160E94131670F3959FC1F3950F50E06F
:102B3000551F629FF001729FBB27F00DB11D639F6F
:102B4000AA27F00DB11DAA1F649F6627B00DA11D15
:102B5000661F829F2227B00DA11D621F739FB00DBB
:102B6000A11D621F839FA00D611D221F749F33272B
:102B7000A00D611D231F849F600D211D822F762FC4
:102B80006A2F11249F5750409AF0F1F088234AF0A1
:102B9000EE0FFF1FBB1F661F771F881F915050400D
:102BA000A9F79E3F510580F00C94EB150C94361656
:102BB0005F3FE4F3983ED4F3869577956795B79594
:102BC000F795E7959F5FC1F7FE2B880F911D9695AE
:102BD000879597F9089597F99F6780E870E060E01E
:102BE00008959FEF80EC089500240A9416161706A6
:102BF00018060906089500240A94121613061406EE
:102C000005060895092E0394000C11F4882352F050
:102C1000BB0F40F4BF2B11F460FF04C06F5F7F4F08
:102C20008F4F9F4F089557FD9058440F551F59F0EF
:102C30005F3F71F04795880F97FB991F61F09F3FA9
:102C400079F087950895121613061406551FF2CFD2
:102C50004695F1DF08C0161617061806991FF1CF22
:102C600086957105610508940895E894BB27662749
:102C70007727CB0197F908950E944716A59F900DDD
:102C8000B49F900DA49F800D911D11240895A29FC3
:102C9000B001B39FC001A39F700D811D1124911D30
:102CA000B29F700D811D1124911D08955058BB27AE
:102CB000AA270E946E160C9402160E94F41538F092
:102CC0000E94FB1520F039F49F3F19F426F40C9470
:102CD000F1150EF4E095E7FB0C94EB15E92F0E943B
:102CE000131658F3BA17620773078407950720F085
:102CF00079F4A6F50C9435160EF4E0950B2EBA2F48
:102D0000A02D0B01B90190010C01CA01A0011124F1
:102D1000FF27591B99F0593F50F4503E68F11A169D
:102D2000F040A22F232F342F4427585FF3CF46952E
:102D300037952795A795F0405395C9F77EF41F1650
:102D4000BA0B620B730B840BBAF09150A1F0FF0F1A
:102D5000BB1F661F771F881FC2F70EC0BA0F621F06
:102D6000731F841F48F4879577956795B795F795F6
:102D70009E3F08F0B0CF9395880F08F09927EE0F8B
:102D80009795879508950E94D7160C9402160E9475
:102D9000FB1558F00E94F41540F029F45F3F29F02C
:102DA0000C94EB1551110C9436160C94F1150E94ED
:102DB000131668F39923B1F3552391F3951B550B23
:102DC000BB27AA2762177307840738F09F5F5F4FFE
:102DD000220F331F441FAA1FA9F335D00E2E3AF03D
:102DE000E0E832D091505040E695001CCAF72BD055
:102DF000FE2F29D0660F771F881FBB1F26173707A6
:102E00004807AB07B0E809F0BB0B802DBF01FF27D7
:102E100093585F4F3AF09E3F510578F00C94EB15B4
:102E20000C9436165F3FE4F3983ED4F3869577957D
:102E30006795B795F7959F5FC9F7880F911D969590
:102E4000879597F90895E1E0660F771F881FBB1FEC
:102E5000621773078407BA0720F0621B730B840B99
:102E6000BA0BEE1F88F7E09508950E943C1768940E
:102E7000B1110C94361608950E941B1688F09F57C6
:102E800098F0B92F9927B751B0F0E1F0660F771F8E
:102E9000881F991F1AF0BA95C9F714C0B13091F084
:102EA0000E943516B1E008950C943516672F782FDF
:102EB0008827B85F39F0B93FCCF386957795679549
:102EC000B395D9F73EF490958095709561957F4FB5
:102ED0008F4F9F4F08950E945A1508F48FEF089561
:102EE0000E945A15880B990B089597FB072E16F42C
:102EF000009407D077FD09D00E94B21707FC05D0D7
:102F00003EF4909581959F4F0895709561957F4F00
:102F10000895A1E21A2EAA1BBB1BFD010DC0AA1F1A
:102F2000BB1FEE1FFF1FA217B307E407F50720F032
:102F3000A21BB30BE40BF50B661F771F881F991FAD
:102F40001A9469F760957095809590959B01AC01F6
:102F5000BD01CF0108950E944716B7FF0895821B57
:102F6000930B0895AA1BBB1B51E107C0AA1FBB1FEF
:102F7000A617B70710F0A61BB70B881F991F5A9505
:102F8000A9F780959095BC01CD010895EE0FFF1F24
:0C2F90000590F491E02D0994F894FFCF17
:102F9C00060909060000000002040E111F100E00A5
:102FAC000A0A111111130D000A0A0E1111110E004B
:102FBC000204111111130D0002040E1111110E0057
:102FCC000204000C04040E0002040E010F110F0089
:102FDC000000A04100C079440000400014005400DF
:102FEC0096008C008000800080006E0069005A0002
:102FFC0050000000000096008C00820078006E00EB
:10300C0064005A005000460000000000E2FFE7FF99
:10301C00ECFFF1FFF6FFFBFF000005000A000F00BC
:10302C0014001C001C00160012000F000C000900FC
:10303C000700050004000300E2FFE7FFECFFF1FFCF
:10304C00F6FFFBFF000005000A000F0014005E00F5
:10305C00BC00770100000000C402F2011F02110342
:10306C0082022E02420200000000E705BA05FD06AE
:10307C009005B305A0059105000000008D09F20133
:10308C00FD0629056E616E00696E66006F7666003E
:10309C0072746563682073797374656D2000732096
:1030AC0076657A00726C002D3E20556A20737A6921
:1030BC006D756C616C7420686F666F6B3A200020C4
:1030CC0043000D0A006E79737A657220497A7A0092
:1030DC0073200020456C00697A7A00733A200073E3
:1030EC0000535A4F4E444120484942412120202050
:1030FC002000204D00643A204B007A6920002041CA
:10310C0075740020496E64007468617400205574F5
:10311C0000204D6F746F722048002052656E6473EE
:0A312C007A6572204B00737A2000D0
:00000001FF
